ARM Linker, 4.1 [Build 713] [Evaluation]

==============================================================================

Section Cross References

    main.o(.text) refers to memcpya.o(.text) for __aeabi_memcpy4
    main.o(.text) refers to mss_gpio.o(.text) for MSS_GPIO_init
    main.o(.text) refers to mss_uart.o(.text) for MSS_UART_init
    main.o(.text) refers to mss_ace.o(.text) for ACE_init
    main.o(.text) refers to ace_convert.o(.text) for ACE_convert_to_mV
    main.o(.text) refers to printf1.o(i.__0snprintf$1) for __2snprintf
    main.o(.text) refers to ace_flags.o(.text) for ACE_get_flag_status
    main.o(.text) refers to mss_uart.o(.bss) for g_mss_uart0
    ace_convert.o(.text) refers to ace_convert.o(.data) for channel_type_lut_h
    ace_convert.o(.text) refers to ace_config.o(.data) for g_ace_channel_desc_table
    ace_convert.o(.text) refers to ace_convert.o(.bss) for g_gdec_lut
    ace_convert.o(.text) refers to ace_convert.o(.constdata) for channel_quad_lut
    ace_convert.o(.text) refers to ace_config.o(.constdata) for g_ace_current_resistors
    ace_flags.o(.text) refers to memcpya.o(.text) for __aeabi_memcpy4
    ace_flags.o(.text) refers to strncmp.o(.text) for strncmp
    ace_flags.o(.text) refers to ace_flags.o(.bss) for g_ppe_flags_isr_lut
    ace_flags.o(.text) refers to ace_config.o(.data) for g_ppe_flags_desc_table
    ace_flags.o(.text) refers to ace_flags.o(.data) for g_ppe_channel_flags_isr_lut
    ace_flags.o(.text) refers to ace_flags.o(.constdata) for .constdata
    mss_ace.o(.text) refers to ace_flags.o(.text) for ace_init_flags
    mss_ace.o(.text) refers to ace_convert.o(.text) for ace_init_convert
    mss_ace.o(.text) refers to mss_ace.o(.constdata) for adc_status_reg_lut
    mss_ace.o(.text) refers to strncmp.o(.text) for strncmp
    mss_ace.o(.text) refers to ace_config.o(.data) for g_ace_channel_desc_table
    mss_gpio.o(.text) refers to mss_gpio.o(.constdata) for g_gpio_irqn_lut
    mss_uart.o(.text) refers to system_a2fxxxm3.o(.text) for SystemCoreClockUpdate
    mss_uart.o(.text) refers to mss_uart.o(.bss) for g_mss_uart0
    mss_uart.o(.text) refers to system_a2fxxxm3.o(.data) for g_FrequencyPCLK0
    system_a2fxxxm3.o(.text) refers to system_a2fxxxm3.o(.constdata) for .constdata
    system_a2fxxxm3.o(.text) refers to system_a2fxxxm3.o(.data) for SystemCoreClock
    ace_config.o(.data) refers to ace_config.o(.constdata) for g_ace_channel_0_name
    entry.o(.ARM.Collect$$$$00000000) refers (Special) to entry7.o(.ARM.Collect$$$$00000007) for _main_init
    entry.o(.ARM.Collect$$$$00000000) refers (Special) to entry5.o(.ARM.Collect$$$$00000004) for _main_scatterload
    entry.o(.ARM.Collect$$$$00000000) refers (Special) to entry2.o(.ARM.Collect$$$$00000001) for _main_stk
    printfb.o(i.__0fprintf$bare) refers to printfb.o(i._printf_core) for _printf_core
    printfb.o(i.__0fprintf$bare) refers to fputc.o(i.fputc) for fputc
    printfb.o(i.__0printf$bare) refers to printfb.o(i._printf_core) for _printf_core
    printfb.o(i.__0printf$bare) refers to fputc.o(i.fputc) for fputc
    printfb.o(i.__0printf$bare) refers to stdout.o(.data) for __stdout
    printfb.o(i.__0snprintf$bare) refers to printfb.o(i._printf_core) for _printf_core
    printfb.o(i.__0snprintf$bare) refers to printfb.o(i._snputc) for _snputc
    printfb.o(i.__0sprintf$bare) refers to printfb.o(i._printf_core) for _printf_core
    printfb.o(i.__0sprintf$bare) refers to printfb.o(i._sputc) for _sputc
    printfb.o(i.__0vfprintf$bare) refers to printfb.o(i._printf_core) for _printf_core
    printfb.o(i.__0vfprintf$bare) refers to fputc.o(i.fputc) for fputc
    printfb.o(i.__0vprintf$bare) refers to printfb.o(i._printf_core) for _printf_core
    printfb.o(i.__0vprintf$bare) refers to fputc.o(i.fputc) for fputc
    printfb.o(i.__0vprintf$bare) refers to stdout.o(.data) for __stdout
    printfb.o(i.__0vsnprintf$bare) refers to printfb.o(i._printf_core) for _printf_core
    printfb.o(i.__0vsnprintf$bare) refers to printfb.o(i._snputc) for _snputc
    printfb.o(i.__0vsprintf$bare) refers to printfb.o(i._printf_core) for _printf_core
    printfb.o(i.__0vsprintf$bare) refers to printfb.o(i._sputc) for _sputc
    printf0.o(i.__0fprintf$0) refers to printf0.o(i._printf_core) for _printf_core
    printf0.o(i.__0fprintf$0) refers to fputc.o(i.fputc) for fputc
    printf0.o(i.__0printf$0) refers to printf0.o(i._printf_core) for _printf_core
    printf0.o(i.__0printf$0) refers to fputc.o(i.fputc) for fputc
    printf0.o(i.__0printf$0) refers to stdout.o(.data) for __stdout
    printf0.o(i.__0snprintf$0) refers to printf0.o(i._printf_core) for _printf_core
    printf0.o(i.__0snprintf$0) refers to printf0.o(i._snputc) for _snputc
    printf0.o(i.__0sprintf$0) refers to printf0.o(i._printf_core) for _printf_core
    printf0.o(i.__0sprintf$0) refers to printf0.o(i._sputc) for _sputc
    printf0.o(i.__0vfprintf$0) refers to printf0.o(i._printf_core) for _printf_core
    printf0.o(i.__0vfprintf$0) refers to fputc.o(i.fputc) for fputc
    printf0.o(i.__0vprintf$0) refers to printf0.o(i._printf_core) for _printf_core
    printf0.o(i.__0vprintf$0) refers to fputc.o(i.fputc) for fputc
    printf0.o(i.__0vprintf$0) refers to stdout.o(.data) for __stdout
    printf0.o(i.__0vsnprintf$0) refers to printf0.o(i._printf_core) for _printf_core
    printf0.o(i.__0vsnprintf$0) refers to printf0.o(i._snputc) for _snputc
    printf0.o(i.__0vsprintf$0) refers to printf0.o(i._printf_core) for _printf_core
    printf0.o(i.__0vsprintf$0) refers to printf0.o(i._sputc) for _sputc
    printf1.o(i.__0fprintf$1) refers to printf1.o(i._printf_core) for _printf_core
    printf1.o(i.__0fprintf$1) refers to fputc.o(i.fputc) for fputc
    printf1.o(i.__0printf$1) refers to printf1.o(i._printf_core) for _printf_core
    printf1.o(i.__0printf$1) refers to fputc.o(i.fputc) for fputc
    printf1.o(i.__0printf$1) refers to stdout.o(.data) for __stdout
    printf1.o(i.__0snprintf$1) refers to printf1.o(i._printf_core) for _printf_core
    printf1.o(i.__0snprintf$1) refers to printf1.o(i._snputc) for _snputc
    printf1.o(i.__0sprintf$1) refers to printf1.o(i._printf_core) for _printf_core
    printf1.o(i.__0sprintf$1) refers to printf1.o(i._sputc) for _sputc
    printf1.o(i.__0vfprintf$1) refers to printf1.o(i._printf_core) for _printf_core
    printf1.o(i.__0vfprintf$1) refers to fputc.o(i.fputc) for fputc
    printf1.o(i.__0vprintf$1) refers to printf1.o(i._printf_core) for _printf_core
    printf1.o(i.__0vprintf$1) refers to fputc.o(i.fputc) for fputc
    printf1.o(i.__0vprintf$1) refers to stdout.o(.data) for __stdout
    printf1.o(i.__0vsnprintf$1) refers to printf1.o(i._printf_core) for _printf_core
    printf1.o(i.__0vsnprintf$1) refers to printf1.o(i._snputc) for _snputc
    printf1.o(i.__0vsprintf$1) refers to printf1.o(i._printf_core) for _printf_core
    printf1.o(i.__0vsprintf$1) refers to printf1.o(i._sputc) for _sputc
    printf1.o(i._printf_core) refers to uidiv.o(.text) for __aeabi_uidivmod
    printf2.o(i.__0fprintf$2) refers to printf2.o(i._printf_core) for _printf_core
    printf2.o(i.__0fprintf$2) refers to fputc.o(i.fputc) for fputc
    printf2.o(i.__0printf$2) refers to printf2.o(i._printf_core) for _printf_core
    printf2.o(i.__0printf$2) refers to fputc.o(i.fputc) for fputc
    printf2.o(i.__0printf$2) refers to stdout.o(.data) for __stdout
    printf2.o(i.__0snprintf$2) refers to printf2.o(i._printf_core) for _printf_core
    printf2.o(i.__0snprintf$2) refers to printf2.o(i._snputc) for _snputc
    printf2.o(i.__0sprintf$2) refers to printf2.o(i._printf_core) for _printf_core
    printf2.o(i.__0sprintf$2) refers to printf2.o(i._sputc) for _sputc
    printf2.o(i.__0vfprintf$2) refers to printf2.o(i._printf_core) for _printf_core
    printf2.o(i.__0vfprintf$2) refers to fputc.o(i.fputc) for fputc
    printf2.o(i.__0vprintf$2) refers to printf2.o(i._printf_core) for _printf_core
    printf2.o(i.__0vprintf$2) refers to fputc.o(i.fputc) for fputc
    printf2.o(i.__0vprintf$2) refers to stdout.o(.data) for __stdout
    printf2.o(i.__0vsnprintf$2) refers to printf2.o(i._printf_core) for _printf_core
    printf2.o(i.__0vsnprintf$2) refers to printf2.o(i._snputc) for _snputc
    printf2.o(i.__0vsprintf$2) refers to printf2.o(i._printf_core) for _printf_core
    printf2.o(i.__0vsprintf$2) refers to printf2.o(i._sputc) for _sputc
    printf3.o(i.__0fprintf$3) refers to printf3.o(i._printf_core) for _printf_core
    printf3.o(i.__0fprintf$3) refers to fputc.o(i.fputc) for fputc
    printf3.o(i.__0printf$3) refers to printf3.o(i._printf_core) for _printf_core
    printf3.o(i.__0printf$3) refers to fputc.o(i.fputc) for fputc
    printf3.o(i.__0printf$3) refers to stdout.o(.data) for __stdout
    printf3.o(i.__0snprintf$3) refers to printf3.o(i._printf_core) for _printf_core
    printf3.o(i.__0snprintf$3) refers to printf3.o(i._snputc) for _snputc
    printf3.o(i.__0sprintf$3) refers to printf3.o(i._printf_core) for _printf_core
    printf3.o(i.__0sprintf$3) refers to printf3.o(i._sputc) for _sputc
    printf3.o(i.__0vfprintf$3) refers to printf3.o(i._printf_core) for _printf_core
    printf3.o(i.__0vfprintf$3) refers to fputc.o(i.fputc) for fputc
    printf3.o(i.__0vprintf$3) refers to printf3.o(i._printf_core) for _printf_core
    printf3.o(i.__0vprintf$3) refers to fputc.o(i.fputc) for fputc
    printf3.o(i.__0vprintf$3) refers to stdout.o(.data) for __stdout
    printf3.o(i.__0vsnprintf$3) refers to printf3.o(i._printf_core) for _printf_core
    printf3.o(i.__0vsnprintf$3) refers to printf3.o(i._snputc) for _snputc
    printf3.o(i.__0vsprintf$3) refers to printf3.o(i._printf_core) for _printf_core
    printf3.o(i.__0vsprintf$3) refers to printf3.o(i._sputc) for _sputc
    printf3.o(i._printf_core) refers to uidiv.o(.text) for __aeabi_uidivmod
    printf4.o(i.__0fprintf$4) refers to printf4.o(i._printf_core) for _printf_core
    printf4.o(i.__0fprintf$4) refers to fputc.o(i.fputc) for fputc
    printf4.o(i.__0printf$4) refers to printf4.o(i._printf_core) for _printf_core
    printf4.o(i.__0printf$4) refers to fputc.o(i.fputc) for fputc
    printf4.o(i.__0printf$4) refers to stdout.o(.data) for __stdout
    printf4.o(i.__0snprintf$4) refers to printf4.o(i._printf_core) for _printf_core
    printf4.o(i.__0snprintf$4) refers to printf4.o(i._snputc) for _snputc
    printf4.o(i.__0sprintf$4) refers to printf4.o(i._printf_core) for _printf_core
    printf4.o(i.__0sprintf$4) refers to printf4.o(i._sputc) for _sputc
    printf4.o(i.__0vfprintf$4) refers to printf4.o(i._printf_core) for _printf_core
    printf4.o(i.__0vfprintf$4) refers to fputc.o(i.fputc) for fputc
    printf4.o(i.__0vprintf$4) refers to printf4.o(i._printf_core) for _printf_core
    printf4.o(i.__0vprintf$4) refers to fputc.o(i.fputc) for fputc
    printf4.o(i.__0vprintf$4) refers to stdout.o(.data) for __stdout
    printf4.o(i.__0vsnprintf$4) refers to printf4.o(i._printf_core) for _printf_core
    printf4.o(i.__0vsnprintf$4) refers to printf4.o(i._snputc) for _snputc
    printf4.o(i.__0vsprintf$4) refers to printf4.o(i._printf_core) for _printf_core
    printf4.o(i.__0vsprintf$4) refers to printf4.o(i._sputc) for _sputc
    printf4.o(i._printf_core) refers to uldiv.o(.text) for __aeabi_uldivmod
    printf5.o(i.__0fprintf$5) refers to printf5.o(i._printf_core) for _printf_core
    printf5.o(i.__0fprintf$5) refers to fputc.o(i.fputc) for fputc
    printf5.o(i.__0printf$5) refers to printf5.o(i._printf_core) for _printf_core
    printf5.o(i.__0printf$5) refers to fputc.o(i.fputc) for fputc
    printf5.o(i.__0printf$5) refers to stdout.o(.data) for __stdout
    printf5.o(i.__0snprintf$5) refers to printf5.o(i._printf_core) for _printf_core
    printf5.o(i.__0snprintf$5) refers to printf5.o(i._snputc) for _snputc
    printf5.o(i.__0sprintf$5) refers to printf5.o(i._printf_core) for _printf_core
    printf5.o(i.__0sprintf$5) refers to printf5.o(i._sputc) for _sputc
    printf5.o(i.__0vfprintf$5) refers to printf5.o(i._printf_core) for _printf_core
    printf5.o(i.__0vfprintf$5) refers to fputc.o(i.fputc) for fputc
    printf5.o(i.__0vprintf$5) refers to printf5.o(i._printf_core) for _printf_core
    printf5.o(i.__0vprintf$5) refers to fputc.o(i.fputc) for fputc
    printf5.o(i.__0vprintf$5) refers to stdout.o(.data) for __stdout
    printf5.o(i.__0vsnprintf$5) refers to printf5.o(i._printf_core) for _printf_core
    printf5.o(i.__0vsnprintf$5) refers to printf5.o(i._snputc) for _snputc
    printf5.o(i.__0vsprintf$5) refers to printf5.o(i._printf_core) for _printf_core
    printf5.o(i.__0vsprintf$5) refers to printf5.o(i._sputc) for _sputc
    printf5.o(i._printf_core) refers to uldiv.o(.text) for __aeabi_uldivmod
    printf6.o(i.__0fprintf$6) refers to printf6.o(i._printf_core) for _printf_core
    printf6.o(i.__0fprintf$6) refers to fputc.o(i.fputc) for fputc
    printf6.o(i.__0printf$6) refers to printf6.o(i._printf_core) for _printf_core
    printf6.o(i.__0printf$6) refers to fputc.o(i.fputc) for fputc
    printf6.o(i.__0printf$6) refers to stdout.o(.data) for __stdout
    printf6.o(i.__0snprintf$6) refers to printf6.o(i._printf_core) for _printf_core
    printf6.o(i.__0snprintf$6) refers to printf6.o(i._snputc) for _snputc
    printf6.o(i.__0sprintf$6) refers to printf6.o(i._printf_core) for _printf_core
    printf6.o(i.__0sprintf$6) refers to printf6.o(i._sputc) for _sputc
    printf6.o(i.__0vfprintf$6) refers to printf6.o(i._printf_core) for _printf_core
    printf6.o(i.__0vfprintf$6) refers to fputc.o(i.fputc) for fputc
    printf6.o(i.__0vprintf$6) refers to printf6.o(i._printf_core) for _printf_core
    printf6.o(i.__0vprintf$6) refers to fputc.o(i.fputc) for fputc
    printf6.o(i.__0vprintf$6) refers to stdout.o(.data) for __stdout
    printf6.o(i.__0vsnprintf$6) refers to printf6.o(i._printf_core) for _printf_core
    printf6.o(i.__0vsnprintf$6) refers to printf6.o(i._snputc) for _snputc
    printf6.o(i.__0vsprintf$6) refers to printf6.o(i._printf_core) for _printf_core
    printf6.o(i.__0vsprintf$6) refers to printf6.o(i._sputc) for _sputc
    printf6.o(i._printf_core) refers to printf6.o(i._printf_pre_padding) for _printf_pre_padding
    printf6.o(i._printf_core) refers to uidiv.o(.text) for __aeabi_uidivmod
    printf6.o(i._printf_core) refers to printf6.o(i._printf_post_padding) for _printf_post_padding
    printf7.o(i.__0fprintf$7) refers to printf7.o(i._printf_core) for _printf_core
    printf7.o(i.__0fprintf$7) refers to fputc.o(i.fputc) for fputc
    printf7.o(i.__0printf$7) refers to printf7.o(i._printf_core) for _printf_core
    printf7.o(i.__0printf$7) refers to fputc.o(i.fputc) for fputc
    printf7.o(i.__0printf$7) refers to stdout.o(.data) for __stdout
    printf7.o(i.__0snprintf$7) refers to printf7.o(i._printf_core) for _printf_core
    printf7.o(i.__0snprintf$7) refers to printf7.o(i._snputc) for _snputc
    printf7.o(i.__0sprintf$7) refers to printf7.o(i._printf_core) for _printf_core
    printf7.o(i.__0sprintf$7) refers to printf7.o(i._sputc) for _sputc
    printf7.o(i.__0vfprintf$7) refers to printf7.o(i._printf_core) for _printf_core
    printf7.o(i.__0vfprintf$7) refers to fputc.o(i.fputc) for fputc
    printf7.o(i.__0vprintf$7) refers to printf7.o(i._printf_core) for _printf_core
    printf7.o(i.__0vprintf$7) refers to fputc.o(i.fputc) for fputc
    printf7.o(i.__0vprintf$7) refers to stdout.o(.data) for __stdout
    printf7.o(i.__0vsnprintf$7) refers to printf7.o(i._printf_core) for _printf_core
    printf7.o(i.__0vsnprintf$7) refers to printf7.o(i._snputc) for _snputc
    printf7.o(i.__0vsprintf$7) refers to printf7.o(i._printf_core) for _printf_core
    printf7.o(i.__0vsprintf$7) refers to printf7.o(i._sputc) for _sputc
    printf7.o(i._printf_core) refers to printf7.o(i._printf_pre_padding) for _printf_pre_padding
    printf7.o(i._printf_core) refers to uldiv.o(.text) for __aeabi_uldivmod
    printf7.o(i._printf_core) refers to printf7.o(i._printf_post_padding) for _printf_post_padding
    printf8.o(i.__0fprintf$8) refers to printf8.o(i._printf_core) for _printf_core
    printf8.o(i.__0fprintf$8) refers to fputc.o(i.fputc) for fputc
    printf8.o(i.__0printf$8) refers to printf8.o(i._printf_core) for _printf_core
    printf8.o(i.__0printf$8) refers to fputc.o(i.fputc) for fputc
    printf8.o(i.__0printf$8) refers to stdout.o(.data) for __stdout
    printf8.o(i.__0snprintf$8) refers to printf8.o(i._printf_core) for _printf_core
    printf8.o(i.__0snprintf$8) refers to printf8.o(i._snputc) for _snputc
    printf8.o(i.__0sprintf$8) refers to printf8.o(i._printf_core) for _printf_core
    printf8.o(i.__0sprintf$8) refers to printf8.o(i._sputc) for _sputc
    printf8.o(i.__0vfprintf$8) refers to printf8.o(i._printf_core) for _printf_core
    printf8.o(i.__0vfprintf$8) refers to fputc.o(i.fputc) for fputc
    printf8.o(i.__0vprintf$8) refers to printf8.o(i._printf_core) for _printf_core
    printf8.o(i.__0vprintf$8) refers to fputc.o(i.fputc) for fputc
    printf8.o(i.__0vprintf$8) refers to stdout.o(.data) for __stdout
    printf8.o(i.__0vsnprintf$8) refers to printf8.o(i._printf_core) for _printf_core
    printf8.o(i.__0vsnprintf$8) refers to printf8.o(i._snputc) for _snputc
    printf8.o(i.__0vsprintf$8) refers to printf8.o(i._printf_core) for _printf_core
    printf8.o(i.__0vsprintf$8) refers to printf8.o(i._sputc) for _sputc
    printf8.o(i._printf_core) refers to printf8.o(i._printf_pre_padding) for _printf_pre_padding
    printf8.o(i._printf_core) refers to uldiv.o(.text) for __aeabi_uldivmod
    printf8.o(i._printf_core) refers to printf8.o(i._printf_post_padding) for _printf_post_padding
    printfa.o(i.__0fprintf) refers (Special) to iusefp.o(.text) for __I$use$fp
    printfa.o(i.__0fprintf) refers to printfa.o(i._printf_core) for _printf_core
    printfa.o(i.__0fprintf) refers to fputc.o(i.fputc) for fputc
    printfa.o(i.__0printf) refers (Special) to iusefp.o(.text) for __I$use$fp
    printfa.o(i.__0printf) refers to printfa.o(i._printf_core) for _printf_core
    printfa.o(i.__0printf) refers to fputc.o(i.fputc) for fputc
    printfa.o(i.__0printf) refers to stdout.o(.data) for __stdout
    printfa.o(i.__0snprintf) refers (Special) to iusefp.o(.text) for __I$use$fp
    printfa.o(i.__0snprintf) refers to printfa.o(i._printf_core) for _printf_core
    printfa.o(i.__0snprintf) refers to printfa.o(i._snputc) for _snputc
    printfa.o(i.__0sprintf) refers (Special) to iusefp.o(.text) for __I$use$fp
    printfa.o(i.__0sprintf) refers to printfa.o(i._printf_core) for _printf_core
    printfa.o(i.__0sprintf) refers to printfa.o(i._sputc) for _sputc
    printfa.o(i.__0vfprintf) refers (Special) to iusefp.o(.text) for __I$use$fp
    printfa.o(i.__0vfprintf) refers to printfa.o(i._printf_core) for _printf_core
    printfa.o(i.__0vfprintf) refers to fputc.o(i.fputc) for fputc
    printfa.o(i.__0vprintf) refers (Special) to iusefp.o(.text) for __I$use$fp
    printfa.o(i.__0vprintf) refers to printfa.o(i._printf_core) for _printf_core
    printfa.o(i.__0vprintf) refers to fputc.o(i.fputc) for fputc
    printfa.o(i.__0vprintf) refers to stdout.o(.data) for __stdout
    printfa.o(i.__0vsnprintf) refers (Special) to iusefp.o(.text) for __I$use$fp
    printfa.o(i.__0vsnprintf) refers to printfa.o(i._printf_core) for _printf_core
    printfa.o(i.__0vsnprintf) refers to printfa.o(i._snputc) for _snputc
    printfa.o(i.__0vsprintf) refers (Special) to iusefp.o(.text) for __I$use$fp
    printfa.o(i.__0vsprintf) refers to printfa.o(i._printf_core) for _printf_core
    printfa.o(i.__0vsprintf) refers to printfa.o(i._sputc) for _sputc
    printfa.o(i._fp_digits) refers (Special) to iusefp.o(.text) for __I$use$fp
    printfa.o(i._fp_digits) refers to dmul.o(.text) for __aeabi_dmul
    printfa.o(i._fp_digits) refers to ddiv.o(.text) for __aeabi_ddiv
    printfa.o(i._fp_digits) refers to cdrcmple.o(.text) for __aeabi_cdrcmple
    printfa.o(i._fp_digits) refers to dadd.o(.text) for __aeabi_dadd
    printfa.o(i._fp_digits) refers to dfixul.o(.text) for __aeabi_d2ulz
    printfa.o(i._fp_digits) refers to uldiv.o(.text) for __aeabi_uldivmod
    printfa.o(i._printf_core) refers (Special) to iusefp.o(.text) for __I$use$fp
    printfa.o(i._printf_core) refers to printfa.o(i._printf_pre_padding) for _printf_pre_padding
    printfa.o(i._printf_core) refers to uldiv.o(.text) for __aeabi_uldivmod
    printfa.o(i._printf_core) refers to printfa.o(i._printf_post_padding) for _printf_post_padding
    printfa.o(i._printf_core) refers to printfa.o(i._fp_digits) for _fp_digits
    printfa.o(i._printf_core) refers to uidiv.o(.text) for __aeabi_uidivmod
    printfa.o(i._printf_post_padding) refers (Special) to iusefp.o(.text) for __I$use$fp
    printfa.o(i._printf_pre_padding) refers (Special) to iusefp.o(.text) for __I$use$fp
    printfa.o(i._snputc) refers (Special) to iusefp.o(.text) for __I$use$fp
    printfa.o(i._sputc) refers (Special) to iusefp.o(.text) for __I$use$fp
    entry2.o(.ARM.Collect$$$$00000001) refers to entry2.o(.ARM.Collect$$$$00002712) for __lit__00000000
    entry2.o(.ARM.Collect$$$$00002712) refers to startup_a2fxxxm3.o(STACK) for __initial_sp
    entry2.o(__vectab_stack_and_reset_area) refers to startup_a2fxxxm3.o(STACK) for __initial_sp
    entry2.o(__vectab_stack_and_reset_area) refers to entry.o(.ARM.Collect$$$$00000000) for __main
    entry5.o(.ARM.Collect$$$$00000004) refers to init.o(.text) for __scatterload
    entry7.o(.ARM.Collect$$$$00000007) refers to main.o(.text) for main
    fputc.o(i.fputc) refers (Special) to iusesemip.o(.text) for __I$use$semihosting$fputc
    fputc.o(i.fputc) refers (Special) to semi.o(.text) for __semihosting_library_function
    uldiv.o(.text) refers to llushr.o(.text) for __aeabi_llsr
    uldiv.o(.text) refers to llshl.o(.text) for __aeabi_llsl
    dadd.o(.text) refers to llshl.o(.text) for __aeabi_llsl
    dadd.o(.text) refers to llsshr.o(.text) for __aeabi_lasr
    dadd.o(.text) refers to depilogue.o(.text) for _double_epilogue
    dmul.o(.text) refers to depilogue.o(.text) for _double_epilogue
    ddiv.o(.text) refers to depilogue.o(.text) for _double_round
    dfixul.o(.text) refers to llushr.o(.text) for __aeabi_llsr
    dfixul.o(.text) refers to llshl.o(.text) for __aeabi_llsl
    startup_a2fxxxm3.o(RESET) refers to startup_a2fxxxm3.o(STACK) for __initial_sp
    startup_a2fxxxm3.o(RESET) refers to startup_a2fxxxm3.o(.text) for Reset_Handler
    startup_a2fxxxm3.o(RESET) refers to mss_uart.o(.text) for UART0_IRQHandler
    startup_a2fxxxm3.o(RESET) refers to ace_flags.o(.text) for ACE_PPE_Flag0_IRQHandler
    startup_a2fxxxm3.o(.text) refers to system_a2fxxxm3.o(.text) for SystemInit
    startup_a2fxxxm3.o(.text) refers to entry.o(.ARM.Collect$$$$00000000) for __main
    init.o(.text) refers to entry5.o(.ARM.Collect$$$$00000004) for __main_after_scatterload
    depilogue.o(.text) refers to llshl.o(.text) for __aeabi_llsl
    depilogue.o(.text) refers to llushr.o(.text) for __aeabi_llsr


==============================================================================

Removing Unused input sections from the image.

    Removing dadd.o(.text), (330 bytes).
    Removing dmul.o(.text), (224 bytes).
    Removing ddiv.o(.text), (222 bytes).
    Removing dfixul.o(.text), (48 bytes).
    Removing cdrcmple.o(.text), (40 bytes).
    Removing startup_a2fxxxm3.o(HEAP), (0 bytes).
    Removing depilogue.o(.text), (194 bytes).

7 unused section(s) (total 1058 bytes) removed from the image.

==============================================================================

Image Symbol Table

    Local Symbols

    Symbol Name                              Value     Ov Type        Size  Object(Section)

    RESET                                    0x00000000   Section      664  startup_a2fxxxm3.o(RESET)
    ../../microlib/division.c                0x00000000   Number         0  uldiv.o ABSOLUTE
    ../../microlib/division.c                0x00000000   Number         0  uidiv.o ABSOLUTE
    ../../microlib/fpadd.c                   0x00000000   Number         0  dadd.o ABSOLUTE
    ../../microlib/fpdiv.c                   0x00000000   Number         0  ddiv.o ABSOLUTE
    ../../microlib/fpepilogue.c              0x00000000   Number         0  depilogue.o ABSOLUTE
    ../../microlib/fpfix.c                   0x00000000   Number         0  dfixul.o ABSOLUTE
    ../../microlib/fpmul.c                   0x00000000   Number         0  dmul.o ABSOLUTE
    ../../microlib/init/entry.s              0x00000000   Number         0  entry5.o ABSOLUTE
    ../../microlib/init/entry.s              0x00000000   Number         0  entry2.o ABSOLUTE
    ../../microlib/init/entry.s              0x00000000   Number         0  entry7.o ABSOLUTE
    ../../microlib/init/entry.s              0x00000000   Number         0  entry.o ABSOLUTE
    ../../microlib/longlong.c                0x00000000   Number         0  llsshr.o ABSOLUTE
    ../../microlib/longlong.c                0x00000000   Number         0  llushr.o ABSOLUTE
    ../../microlib/longlong.c                0x00000000   Number         0  llshl.o ABSOLUTE
    ../../microlib/printf/printf.c           0x00000000   Number         0  printf5.o ABSOLUTE
    ../../microlib/printf/printf.c           0x00000000   Number         0  printf1.o ABSOLUTE
    ../../microlib/printf/printf.c           0x00000000   Number         0  printfa.o ABSOLUTE
    ../../microlib/printf/printf.c           0x00000000   Number         0  printf8.o ABSOLUTE
    ../../microlib/printf/printf.c           0x00000000   Number         0  printf7.o ABSOLUTE
    ../../microlib/printf/printf.c           0x00000000   Number         0  printf6.o ABSOLUTE
    ../../microlib/printf/printf.c           0x00000000   Number         0  printf0.o ABSOLUTE
    ../../microlib/printf/printf.c           0x00000000   Number         0  printfb.o ABSOLUTE
    ../../microlib/printf/printf.c           0x00000000   Number         0  printf4.o ABSOLUTE
    ../../microlib/printf/printf.c           0x00000000   Number         0  printf3.o ABSOLUTE
    ../../microlib/printf/printf.c           0x00000000   Number         0  printf2.o ABSOLUTE
    ../../microlib/printf/stubs.s            0x00000000   Number         0  stubs.o ABSOLUTE
    ../../microlib/stdio/fputc.c             0x00000000   Number         0  fputc.o ABSOLUTE
    ../../microlib/stdio/semi.s              0x00000000   Number         0  semi.o ABSOLUTE
    ../../microlib/stdio/streams.c           0x00000000   Number         0  stdout.o ABSOLUTE
    ../../microlib/string/memcpy.c           0x00000000   Number         0  memcpyb.o ABSOLUTE
    ../../microlib/string/memcpy.c           0x00000000   Number         0  memcpya.o ABSOLUTE
    ../../microlib/string/strncmp.c          0x00000000   Number         0  strncmp.o ABSOLUTE
    ../../microlib/stubs.s                   0x00000000   Number         0  iusefp.o ABSOLUTE
    ../../microlib/stubs.s                   0x00000000   Number         0  iusesemip.o ABSOLUTE
    CMSIS/startup_arm/startup_a2fxxxm3.s     0x00000000   Number         0  startup_a2fxxxm3.o ABSOLUTE
    CMSIS/system_a2fxxxm3.c                  0x00000000   Number         0  system_a2fxxxm3.o ABSOLUTE
    cdrcmple.s                               0x00000000   Number         0  cdrcmple.o ABSOLUTE
    dc.s                                     0x00000000   Number         0  dc.o ABSOLUTE
    drivers/mss_ace/ace_convert.c            0x00000000   Number         0  ace_convert.o ABSOLUTE
    drivers/mss_ace/ace_flags.c              0x00000000   Number         0  ace_flags.o ABSOLUTE
    drivers/mss_ace/mss_ace.c                0x00000000   Number         0  mss_ace.o ABSOLUTE
    drivers/mss_gpio/mss_gpio.c              0x00000000   Number         0  mss_gpio.o ABSOLUTE
    drivers/mss_uart/mss_uart.c              0x00000000   Number         0  mss_uart.o ABSOLUTE
    drivers_config/mss_ace/ace_config.c      0x00000000   Number         0  ace_config.o ABSOLUTE
    handlers.s                               0x00000000   Number         0  handlers.o ABSOLUTE
    init.s                                   0x00000000   Number         0  init.o ABSOLUTE
    main.c                                   0x00000000   Number         0  main.o ABSOLUTE
    .ARM.Collect$$$$00000000                 0x00000298   Section        0  entry.o(.ARM.Collect$$$$00000000)
    .ARM.Collect$$$$00000001                 0x00000298   Section        4  entry2.o(.ARM.Collect$$$$00000001)
    .ARM.Collect$$$$00000004                 0x0000029c   Section        4  entry5.o(.ARM.Collect$$$$00000004)
    .ARM.Collect$$$$00000007                 0x000002a0   Section        8  entry7.o(.ARM.Collect$$$$00000007)
    .ARM.Collect$$$$00002712                 0x000002a8   Section        4  entry2.o(.ARM.Collect$$$$00002712)
    __lit__00000000                          0x000002a8   Data           4  entry2.o(.ARM.Collect$$$$00002712)
    .text                                    0x000002ac   Section        0  main.o(.text)
    .text                                    0x00000464   Section        0  ace_convert.o(.text)
    convert_mV_to_ppe_value                  0x0000075b   Thumb Code    54  ace_convert.o(.text)
    .text                                    0x000009c8   Section        0  ace_flags.o(.text)
    process_flag_irq                         0x00000ffb   Thumb Code   184  ace_flags.o(.text)
    NVIC_ClearPendingIRQ                     0x000012dd   Thumb Code    24  ace_flags.o(.text)
    .text                                    0x000012f8   Section        0  mss_ace.o(.text)
    .text                                    0x00001894   Section        0  mss_gpio.o(.text)
    NVIC_ClearPendingIRQ                     0x000019f9   Thumb Code    24  mss_gpio.o(.text)
    .text                                    0x00001a30   Section        0  mss_uart.o(.text)
    default_tx_handler                       0x00001a31   Thumb Code   116  mss_uart.o(.text)
    MSS_UART_isr                             0x00001d95   Thumb Code   104  mss_uart.o(.text)
    NVIC_EnableIRQ                           0x00002003   Thumb Code    30  mss_uart.o(.text)
    NVIC_ClearPendingIRQ                     0x00002021   Thumb Code    24  mss_uart.o(.text)
    .text                                    0x00002044   Section        0  system_a2fxxxm3.o(.text)
    GetSystemClock                           0x00002047   Thumb Code    88  system_a2fxxxm3.o(.text)
    .text                                    0x00002174   Section        0  memcpya.o(.text)
    .text                                    0x00002198   Section        0  strncmp.o(.text)
    .text                                    0x000021b6   Section        0  uidiv.o(.text)
    .text                                    0x000021e4   Section       36  startup_a2fxxxm3.o(.text)
    .text                                    0x00002208   Section       36  init.o(.text)
    i.__0snprintf$1                          0x0000222c   Section        0  printf1.o(i.__0snprintf$1)
    i.__scatterload_copy                     0x00002254   Section       14  handlers.o(i.__scatterload_copy)
    i.__scatterload_null                     0x00002262   Section        2  handlers.o(i.__scatterload_null)
    i.__scatterload_zeroinit                 0x00002264   Section       14  handlers.o(i.__scatterload_zeroinit)
    i._printf_core                           0x00002274   Section        0  printf1.o(i._printf_core)
    _printf_core                             0x00002275   Thumb Code   332  printf1.o(i._printf_core)
    i._snputc                                0x000023c4   Section        0  printf1.o(i._snputc)
    _snputc                                  0x000023c5   Thumb Code    22  printf1.o(i._snputc)
    .constdata                               0x000023da   Section      204  ace_convert.o(.constdata)
    channel_type_lut                         0x000023da   Data          48  ace_convert.o(.constdata)
    channel_quad_lut                         0x0000240a   Data          48  ace_convert.o(.constdata)
    abps_channel_lut                         0x0000243a   Data          48  ace_convert.o(.constdata)
    abps_idx_lut                             0x0000246a   Data          48  ace_convert.o(.constdata)
    apbs_gain_lut                            0x0000249a   Data           4  ace_convert.o(.constdata)
    apbs_range                               0x0000249e   Data           8  ace_convert.o(.constdata)
    .constdata                               0x000024a8   Section      176  ace_flags.o(.constdata)
    g_ppe_flags_regs_lut                     0x000024a8   Data          20  ace_flags.o(.constdata)
    flags_irq_enable_regs_lut                0x000024bc   Data          20  ace_flags.o(.constdata)
    flags_irq_status_regs_lut                0x000024d0   Data          20  ace_flags.o(.constdata)
    flags_irq_clear_regs_lut                 0x000024e4   Data          20  ace_flags.o(.constdata)
    threshold_irqn_lut                       0x000024f8   Data          64  ace_flags.o(.constdata)
    .constdata                               0x00002558   Section       70  mss_ace.o(.constdata)
    adc_status_reg_lut                       0x00002558   Data          12  mss_ace.o(.constdata)
    dac_ctrl_reg_lut                         0x00002564   Data          12  mss_ace.o(.constdata)
    dac_enable_masks_lut                     0x00002570   Data          12  mss_ace.o(.constdata)
    dac_byte01_reg_lut                       0x0000257c   Data          12  mss_ace.o(.constdata)
    dac_byte2_reg_lut                        0x00002588   Data          12  mss_ace.o(.constdata)
    .constdata                               0x000025a0   Section      192  mss_gpio.o(.constdata)
    g_config_reg_lut                         0x000025a0   Data         128  mss_gpio.o(.constdata)
    g_gpio_irqn_lut                          0x00002620   Data          64  mss_gpio.o(.constdata)
    .constdata                               0x00002660   Section       16  system_a2fxxxm3.o(.constdata)
    .constdata                               0x00002670   Section      164  ace_config.o(.constdata)
    .data                                    0x20000000   Section        1  ace_convert.o(.data)
    channel_type_lut_h                       0x20000000   Data           1  ace_convert.o(.data)
    .data                                    0x20000004   Section        8  ace_flags.o(.data)
    g_ppe_global_flags_isr                   0x20000004   Data           4  ace_flags.o(.data)
    g_ppe_channel_flags_isr_lut              0x20000008   Data           4  ace_flags.o(.data)
    .data                                    0x2000000c   Section       24  system_a2fxxxm3.o(.data)
    .data                                    0x20000024   Section      128  ace_config.o(.data)
    .bss                                     0x200000a4   Section       10  ace_convert.o(.bss)
    g_gdec_lut                               0x200000a4   Data          10  ace_convert.o(.bss)
    .bss                                     0x200000b0   Section      800  ace_flags.o(.bss)
    g_ppe_flag_handles_lut                   0x200000b0   Data         160  ace_flags.o(.bss)
    g_ppe_flags_isr_lut                      0x20000150   Data         640  ace_flags.o(.bss)
    .bss                                     0x200003d0   Section       80  mss_uart.o(.bss)
    STACK                                    0x20000420   Section     4096  startup_a2fxxxm3.o(STACK)

    Global Symbols

    Symbol Name                              Value     Ov Type        Size  Object(Section)

    BuildAttributes$$THM_ISAv4$P$D$K$B$S$PE$A:L22UL41UL21$X:L11$S22US41US21$IEEE1$IW$USESV6$~STKCKD$USESV7$~SHL$OSPACE$ROPI$EBA8$MICROLIB$REQ8$PRES8$EABIv2 0x00000000   Number         0  anon$$obj.o ABSOLUTE
    __ARM_use_no_argv                        0x00000000   Number         0  main.o ABSOLUTE
    __Vectors                                0x00000000   Data           4  startup_a2fxxxm3.o(RESET)
    _printf_a                                0x00000000   Number         0  stubs.o ABSOLUTE
    _printf_c                                0x00000000   Number         0  stubs.o ABSOLUTE
    _printf_charcount                        0x00000000   Number         0  stubs.o ABSOLUTE
    _printf_d                                0x00000000   Number         0  stubs.o ABSOLUTE
    _printf_e                                0x00000000   Number         0  stubs.o ABSOLUTE
    _printf_f                                0x00000000   Number         0  stubs.o ABSOLUTE
    _printf_flags                            0x00000000   Number         0  stubs.o ABSOLUTE
    _printf_fp_dec                           0x00000000   Number         0  stubs.o ABSOLUTE
    _printf_fp_hex                           0x00000000   Number         0  stubs.o ABSOLUTE
    _printf_g                                0x00000000   Number         0  stubs.o ABSOLUTE
    _printf_i                                0x00000000   Number         0  stubs.o ABSOLUTE
    _printf_int_dec                          0x00000000   Number         0  stubs.o ABSOLUTE
    _printf_l                                0x00000000   Number         0  stubs.o ABSOLUTE
    _printf_lc                               0x00000000   Number         0  stubs.o ABSOLUTE
    _printf_ll                               0x00000000   Number         0  stubs.o ABSOLUTE
    _printf_lld                              0x00000000   Number         0  stubs.o ABSOLUTE
    _printf_lli                              0x00000000   Number         0  stubs.o ABSOLUTE
    _printf_llo                              0x00000000   Number         0  stubs.o ABSOLUTE
    _printf_llu                              0x00000000   Number         0  stubs.o ABSOLUTE
    _printf_llx                              0x00000000   Number         0  stubs.o ABSOLUTE
    _printf_longlong_dec                     0x00000000   Number         0  stubs.o ABSOLUTE
    _printf_longlong_hex                     0x00000000   Number         0  stubs.o ABSOLUTE
    _printf_longlong_oct                     0x00000000   Number         0  stubs.o ABSOLUTE
    _printf_ls                               0x00000000   Number         0  stubs.o ABSOLUTE
    _printf_mbtowc                           0x00000000   Number         0  stubs.o ABSOLUTE
    _printf_n                                0x00000000   Number         0  stubs.o ABSOLUTE
    _printf_o                                0x00000000   Number         0  stubs.o ABSOLUTE
    _printf_p                                0x00000000   Number         0  stubs.o ABSOLUTE
    _printf_percent                          0x00000000   Number         0  stubs.o ABSOLUTE
    _printf_pre_padding                      0x00000000   Number         0  stubs.o ABSOLUTE
    _printf_return_value                     0x00000000   Number         0  stubs.o ABSOLUTE
    _printf_s                                0x00000000   Number         0  stubs.o ABSOLUTE
    _printf_sizespec                         0x00000000   Number         0  stubs.o ABSOLUTE
    _printf_str                              0x00000000   Number         0  stubs.o ABSOLUTE
    _printf_truncate_signed                  0x00000000   Number         0  stubs.o ABSOLUTE
    _printf_truncate_unsigned                0x00000000   Number         0  stubs.o ABSOLUTE
    _printf_u                                0x00000000   Number         0  stubs.o ABSOLUTE
    _printf_wc                               0x00000000   Number         0  stubs.o ABSOLUTE
    _printf_wctomb                           0x00000000   Number         0  stubs.o ABSOLUTE
    _printf_widthprec                        0x00000000   Number         0  stubs.o ABSOLUTE
    _printf_x                                0x00000000   Number         0  stubs.o ABSOLUTE
    __decompress                              - Undefined Weak Reference
    __Vectors_End                            0x00000298   Data           0  startup_a2fxxxm3.o(RESET)
    __Vectors_Size                           0x00000298   Number         0  startup_a2fxxxm3.o ABSOLUTE
    __main                                   0x00000299   Thumb Code     0  entry.o(.ARM.Collect$$$$00000000)
    _main_stk                                0x00000299   Thumb Code     0  entry2.o(.ARM.Collect$$$$00000001)
    _main_scatterload                        0x0000029d   Thumb Code     0  entry5.o(.ARM.Collect$$$$00000004)
    __main_after_scatterload                 0x000002a1   Thumb Code     0  entry5.o(.ARM.Collect$$$$00000004)
    _main_init                               0x000002a1   Thumb Code     0  entry7.o(.ARM.Collect$$$$00000007)
    main                                     0x000002ad   Thumb Code   332  main.o(.text)
    ACE_get_channel_type                     0x00000465   Thumb Code    22  ace_convert.o(.text)
    ACE_convert_adc_input_to_mV              0x0000047b   Thumb Code    40  ace_convert.o(.text)
    ace_init_convert                         0x000004a3   Thumb Code   202  ace_convert.o(.text)
    ACE_convert_to_mV                        0x0000056d   Thumb Code   126  ace_convert.o(.text)
    ACE_convert_to_mA                        0x000005eb   Thumb Code    86  ace_convert.o(.text)
    ACE_convert_to_uA                        0x00000641   Thumb Code    86  ace_convert.o(.text)
    ACE_convert_to_Kelvin                    0x00000697   Thumb Code    36  ace_convert.o(.text)
    ACE_convert_to_Celsius                   0x000006bb   Thumb Code    28  ace_convert.o(.text)
    ACE_convert_to_Fahrenheit                0x000006d7   Thumb Code    36  ace_convert.o(.text)
    ACE_get_channel_name                     0x000006fb   Thumb Code    20  ace_convert.o(.text)
    ACE_convert_mV_to_adc_value              0x0000070f   Thumb Code    76  ace_convert.o(.text)
    ACE_convert_from_mV                      0x00000791   Thumb Code   146  ace_convert.o(.text)
    ACE_convert_from_mA                      0x00000823   Thumb Code   154  ace_convert.o(.text)
    ACE_convert_from_uA                      0x000008bd   Thumb Code    96  ace_convert.o(.text)
    ACE_convert_from_Kelvin                  0x0000091d   Thumb Code    50  ace_convert.o(.text)
    ACE_convert_from_Celsius                 0x0000094f   Thumb Code    42  ace_convert.o(.text)
    ACE_convert_from_Fahrenheit              0x00000979   Thumb Code    52  ace_convert.o(.text)
    ACE_translate_pdma_value                 0x000009ad   Thumb Code    16  ace_convert.o(.text)
    ace_init_flags                           0x000009c9   Thumb Code    98  ace_flags.o(.text)
    ACE_is_hysteresis_flag                   0x00000a2b   Thumb Code    24  ace_flags.o(.text)
    ACE_is_under_flag                        0x00000a43   Thumb Code    52  ace_flags.o(.text)
    ACE_set_flag_threshold                   0x00000a77   Thumb Code   220  ace_flags.o(.text)
    ACE_set_flag_assertion                   0x00000b53   Thumb Code    88  ace_flags.o(.text)
    ACE_set_flag_deassertion                 0x00000bab   Thumb Code    80  ace_flags.o(.text)
    ACE_set_flag_hysteresis                  0x00000bfb   Thumb Code   164  ace_flags.o(.text)
    ACE_set_channel_hysteresis               0x00000c9f   Thumb Code    60  ace_flags.o(.text)
    ACE_get_flag_handle                      0x00000cdb   Thumb Code    70  ace_flags.o(.text)
    ACE_get_flag_status                      0x00000d21   Thumb Code    72  ace_flags.o(.text)
    ACE_get_flag_name                        0x00000d69   Thumb Code    20  ace_flags.o(.text)
    ACE_get_flag_channel                     0x00000d7d   Thumb Code    20  ace_flags.o(.text)
    ACE_get_channel_flag_count               0x00000d91   Thumb Code    20  ace_flags.o(.text)
    ACE_get_channel_first_flag               0x00000da5   Thumb Code    88  ace_flags.o(.text)
    ACE_get_channel_next_flag                0x00000dfd   Thumb Code    68  ace_flags.o(.text)
    ACE_enable_flag_irq                      0x00000e41   Thumb Code    94  ace_flags.o(.text)
    ACE_enable_channel_flags_irq             0x00000e9f   Thumb Code    52  ace_flags.o(.text)
    ACE_disable_flag_irq                     0x00000ed3   Thumb Code    74  ace_flags.o(.text)
    ACE_disable_channel_flags_irq            0x00000f1d   Thumb Code    52  ace_flags.o(.text)
    ACE_clear_flag_irq                       0x00000f51   Thumb Code    74  ace_flags.o(.text)
    ACE_clear_channel_flags_irq              0x00000f9b   Thumb Code    52  ace_flags.o(.text)
    ACE_register_flag_isr                    0x00000fcf   Thumb Code    26  ace_flags.o(.text)
    ACE_register_channel_flags_isr           0x00000fe9   Thumb Code    12  ace_flags.o(.text)
    ACE_register_global_flags_isr            0x00000ff5   Thumb Code     6  ace_flags.o(.text)
    ACE_PPE_Flag0_IRQHandler                 0x000010b3   Thumb Code    16  ace_flags.o(.text)
    ACE_PPE_Flag1_IRQHandler                 0x000010c3   Thumb Code    16  ace_flags.o(.text)
    ACE_PPE_Flag2_IRQHandler                 0x000010d3   Thumb Code    16  ace_flags.o(.text)
    ACE_PPE_Flag3_IRQHandler                 0x000010e3   Thumb Code    16  ace_flags.o(.text)
    ACE_PPE_Flag4_IRQHandler                 0x000010f3   Thumb Code    16  ace_flags.o(.text)
    ACE_PPE_Flag5_IRQHandler                 0x00001103   Thumb Code    16  ace_flags.o(.text)
    ACE_PPE_Flag6_IRQHandler                 0x00001113   Thumb Code    16  ace_flags.o(.text)
    ACE_PPE_Flag7_IRQHandler                 0x00001123   Thumb Code    16  ace_flags.o(.text)
    ACE_PPE_Flag8_IRQHandler                 0x00001133   Thumb Code    16  ace_flags.o(.text)
    ACE_PPE_Flag9_IRQHandler                 0x00001143   Thumb Code    16  ace_flags.o(.text)
    ACE_PPE_Flag10_IRQHandler                0x00001153   Thumb Code    16  ace_flags.o(.text)
    ACE_PPE_Flag11_IRQHandler                0x00001163   Thumb Code    16  ace_flags.o(.text)
    ACE_PPE_Flag12_IRQHandler                0x00001173   Thumb Code    16  ace_flags.o(.text)
    ACE_PPE_Flag13_IRQHandler                0x00001183   Thumb Code    16  ace_flags.o(.text)
    ACE_PPE_Flag14_IRQHandler                0x00001193   Thumb Code    16  ace_flags.o(.text)
    ACE_PPE_Flag15_IRQHandler                0x000011a3   Thumb Code    16  ace_flags.o(.text)
    ACE_PPE_Flag16_IRQHandler                0x000011b3   Thumb Code    16  ace_flags.o(.text)
    ACE_PPE_Flag17_IRQHandler                0x000011c3   Thumb Code    16  ace_flags.o(.text)
    ACE_PPE_Flag18_IRQHandler                0x000011d3   Thumb Code    16  ace_flags.o(.text)
    ACE_PPE_Flag19_IRQHandler                0x000011e3   Thumb Code    58  ace_flags.o(.text)
    ACE_PPE_Flag20_IRQHandler                0x0000121d   Thumb Code    16  ace_flags.o(.text)
    ACE_PPE_Flag21_IRQHandler                0x0000122d   Thumb Code    16  ace_flags.o(.text)
    ACE_PPE_Flag22_IRQHandler                0x0000123d   Thumb Code    16  ace_flags.o(.text)
    ACE_PPE_Flag23_IRQHandler                0x0000124d   Thumb Code    16  ace_flags.o(.text)
    ACE_PPE_Flag24_IRQHandler                0x0000125d   Thumb Code    16  ace_flags.o(.text)
    ACE_PPE_Flag25_IRQHandler                0x0000126d   Thumb Code    16  ace_flags.o(.text)
    ACE_PPE_Flag26_IRQHandler                0x0000127d   Thumb Code    16  ace_flags.o(.text)
    ACE_PPE_Flag27_IRQHandler                0x0000128d   Thumb Code    16  ace_flags.o(.text)
    ACE_PPE_Flag28_IRQHandler                0x0000129d   Thumb Code    16  ace_flags.o(.text)
    ACE_PPE_Flag29_IRQHandler                0x000012ad   Thumb Code    16  ace_flags.o(.text)
    ACE_PPE_Flag30_IRQHandler                0x000012bd   Thumb Code    16  ace_flags.o(.text)
    ACE_PPE_Flag31_IRQHandler                0x000012cd   Thumb Code    16  ace_flags.o(.text)
    ACE_init                                 0x000012f9   Thumb Code    12  mss_ace.o(.text)
    ACE_start_adc                            0x00001305   Thumb Code    10  mss_ace.o(.text)
    ACE_get_adc_result                       0x0000130f   Thumb Code    42  mss_ace.o(.text)
    ACE_configure_sdd                        0x00001339   Thumb Code   234  mss_ace.o(.text)
    ACE_enable_sdd                           0x00001423   Thumb Code    26  mss_ace.o(.text)
    ACE_disable_sdd                          0x0000143d   Thumb Code    26  mss_ace.o(.text)
    ACE_set_sdd_value                        0x00001457   Thumb Code    26  mss_ace.o(.text)
    ACE_set_sdd_value_sync                   0x00001471   Thumb Code    88  mss_ace.o(.text)
    ACE_set_comp_reference                   0x000014c9   Thumb Code   184  mss_ace.o(.text)
    ACE_set_comp_hysteresis                  0x00001581   Thumb Code   126  mss_ace.o(.text)
    ACE_enable_comp                          0x000015ff   Thumb Code   106  mss_ace.o(.text)
    ACE_disable_comp                         0x00001669   Thumb Code   106  mss_ace.o(.text)
    ACE_enable_comp_rise_irq                 0x000016d3   Thumb Code    98  mss_ace.o(.text)
    ACE_disable_comp_rise_irq                0x00001735   Thumb Code    32  mss_ace.o(.text)
    ACE_clear_comp_rise_irq                  0x00001755   Thumb Code    32  mss_ace.o(.text)
    ACE_enable_comp_fall_irq                 0x00001775   Thumb Code    24  mss_ace.o(.text)
    ACE_disable_comp_fall_irq                0x0000178d   Thumb Code    32  mss_ace.o(.text)
    ACE_clear_comp_fall_irq                  0x000017ad   Thumb Code    32  mss_ace.o(.text)
    ACE_get_comp_status                      0x000017cd   Thumb Code     6  mss_ace.o(.text)
    ACE_get_channel_count                    0x000017d3   Thumb Code     4  mss_ace.o(.text)
    ACE_get_first_channel                    0x000017d7   Thumb Code     6  mss_ace.o(.text)
    ACE_get_next_channel                     0x000017dd   Thumb Code    16  mss_ace.o(.text)
    ACE_get_channel_handle                   0x000017ed   Thumb Code    70  mss_ace.o(.text)
    ACE_get_input_channel_handle             0x00001833   Thumb Code    42  mss_ace.o(.text)
    ACE_get_ppe_sample                       0x0000185d   Thumb Code    32  mss_ace.o(.text)
    MSS_GPIO_init                            0x00001895   Thumb Code    52  mss_gpio.o(.text)
    MSS_GPIO_config                          0x000018c9   Thumb Code    16  mss_gpio.o(.text)
    MSS_GPIO_set_output                      0x000018d9   Thumb Code    14  mss_gpio.o(.text)
    MSS_GPIO_drive_inout                     0x000018e7   Thumb Code   140  mss_gpio.o(.text)
    MSS_GPIO_enable_irq                      0x00001973   Thumb Code    70  mss_gpio.o(.text)
    MSS_GPIO_disable_irq                     0x000019b9   Thumb Code    30  mss_gpio.o(.text)
    MSS_GPIO_clear_irq                       0x000019d7   Thumb Code    34  mss_gpio.o(.text)
    MSS_UART_init                            0x00001aa5   Thumb Code   266  mss_uart.o(.text)
    MSS_UART_polled_tx                       0x00001baf   Thumb Code    94  mss_uart.o(.text)
    MSS_UART_polled_tx_string                0x00001c0d   Thumb Code    76  mss_uart.o(.text)
    MSS_UART_irq_tx                          0x00001c59   Thumb Code    66  mss_uart.o(.text)
    MSS_UART_tx_complete                     0x00001c9b   Thumb Code    48  mss_uart.o(.text)
    MSS_UART_get_rx                          0x00001ccb   Thumb Code    74  mss_uart.o(.text)
    MSS_UART_enable_irq                      0x00001d15   Thumb Code    48  mss_uart.o(.text)
    MSS_UART_disable_irq                     0x00001d45   Thumb Code    80  mss_uart.o(.text)
    MSS_UART_set_rx_handler                  0x00001dfd   Thumb Code   108  mss_uart.o(.text)
    MSS_UART_set_loopback                    0x00001e69   Thumb Code    38  mss_uart.o(.text)
    UART0_IRQHandler                         0x00001e8f   Thumb Code    16  mss_uart.o(.text)
    UART1_IRQHandler                         0x00001e9f   Thumb Code    16  mss_uart.o(.text)
    MSS_UART_set_rxstatus_handler            0x00001eaf   Thumb Code    50  mss_uart.o(.text)
    MSS_UART_set_tx_handler                  0x00001ee1   Thumb Code    58  mss_uart.o(.text)
    MSS_UART_set_modemstatus_handler         0x00001f1b   Thumb Code    50  mss_uart.o(.text)
    MSS_UART_fill_tx_fifo                    0x00001f4d   Thumb Code    78  mss_uart.o(.text)
    MSS_UART_get_rx_status                   0x00001f9b   Thumb Code    44  mss_uart.o(.text)
    MSS_UART_get_modem_status                0x00001fc7   Thumb Code    24  mss_uart.o(.text)
    MSS_UART_get_tx_status                   0x00001fdf   Thumb Code    36  mss_uart.o(.text)
    SystemInit                               0x00002045   Thumb Code     2  system_a2fxxxm3.o(.text)
    SystemCoreClockUpdate                    0x0000209f   Thumb Code   142  system_a2fxxxm3.o(.text)
    __aeabi_memcpy                           0x00002175   Thumb Code    36  memcpya.o(.text)
    __aeabi_memcpy4                          0x00002175   Thumb Code     0  memcpya.o(.text)
    __aeabi_memcpy8                          0x00002175   Thumb Code     0  memcpya.o(.text)
    strncmp                                  0x00002199   Thumb Code    30  strncmp.o(.text)
    __aeabi_uidiv                            0x000021b7   Thumb Code     0  uidiv.o(.text)
    __aeabi_uidivmod                         0x000021b7   Thumb Code    44  uidiv.o(.text)
    Reset_Handler                            0x000021e5   Thumb Code     8  startup_a2fxxxm3.o(.text)
    NMI_Handler                              0x000021ed   Thumb Code     2  startup_a2fxxxm3.o(.text)
    HardFault_Handler                        0x000021ef   Thumb Code     2  startup_a2fxxxm3.o(.text)
    MemManage_Handler                        0x000021f1   Thumb Code     2  startup_a2fxxxm3.o(.text)
    BusFault_Handler                         0x000021f3   Thumb Code     2  startup_a2fxxxm3.o(.text)
    UsageFault_Handler                       0x000021f5   Thumb Code     2  startup_a2fxxxm3.o(.text)
    SVC_Handler                              0x000021f7   Thumb Code     2  startup_a2fxxxm3.o(.text)
    DebugMon_Handler                         0x000021f9   Thumb Code     2  startup_a2fxxxm3.o(.text)
    PendSV_Handler                           0x000021fb   Thumb Code     2  startup_a2fxxxm3.o(.text)
    SysTick_Handler                          0x000021fd   Thumb Code     2  startup_a2fxxxm3.o(.text)
    ACE_ADC0_CalDone_IRQHandler              0x000021ff   Thumb Code     0  startup_a2fxxxm3.o(.text)
    ACE_ADC0_CalStart_IRQHandler             0x000021ff   Thumb Code     0  startup_a2fxxxm3.o(.text)
    ACE_ADC0_DataValid_IRQHandler            0x000021ff   Thumb Code     0  startup_a2fxxxm3.o(.text)
    ACE_ADC0_FifoAFull_IRQHandler            0x000021ff   Thumb Code     0  startup_a2fxxxm3.o(.text)
    ACE_ADC0_FifoEmpty_IRQHandler            0x000021ff   Thumb Code     0  startup_a2fxxxm3.o(.text)
    ACE_ADC0_FifoFull_IRQHandler             0x000021ff   Thumb Code     0  startup_a2fxxxm3.o(.text)
    ACE_ADC1_CalDone_IRQHandler              0x000021ff   Thumb Code     0  startup_a2fxxxm3.o(.text)
    ACE_ADC1_CalStart_IRQHandler             0x000021ff   Thumb Code     0  startup_a2fxxxm3.o(.text)
    ACE_ADC1_DataValid_IRQHandler            0x000021ff   Thumb Code     0  startup_a2fxxxm3.o(.text)
    ACE_ADC1_FifoAFull_IRQHandler            0x000021ff   Thumb Code     0  startup_a2fxxxm3.o(.text)
    ACE_ADC1_FifoEmpty_IRQHandler            0x000021ff   Thumb Code     0  startup_a2fxxxm3.o(.text)
    ACE_ADC1_FifoFull_IRQHandler             0x000021ff   Thumb Code     0  startup_a2fxxxm3.o(.text)
    ACE_ADC2_CalDone_IRQHandler              0x000021ff   Thumb Code     0  startup_a2fxxxm3.o(.text)
    ACE_ADC2_CalStart_IRQHandler             0x000021ff   Thumb Code     0  startup_a2fxxxm3.o(.text)
    ACE_ADC2_DataValid_IRQHandler            0x000021ff   Thumb Code     0  startup_a2fxxxm3.o(.text)
    ACE_ADC2_FifoAFull_IRQHandler            0x000021ff   Thumb Code     0  startup_a2fxxxm3.o(.text)
    ACE_ADC2_FifoEmpty_IRQHandler            0x000021ff   Thumb Code     0  startup_a2fxxxm3.o(.text)
    ACE_ADC2_FifoFull_IRQHandler             0x000021ff   Thumb Code     0  startup_a2fxxxm3.o(.text)
    ACE_Comp0_Fall_IRQHandler                0x000021ff   Thumb Code     0  startup_a2fxxxm3.o(.text)
    ACE_Comp0_Rise_IRQHandler                0x000021ff   Thumb Code     0  startup_a2fxxxm3.o(.text)
    ACE_Comp10_Fall_IRQHandler               0x000021ff   Thumb Code     0  startup_a2fxxxm3.o(.text)
    ACE_Comp10_Rise_IRQHandler               0x000021ff   Thumb Code     0  startup_a2fxxxm3.o(.text)
    ACE_Comp11_Fall_IRQHandler               0x000021ff   Thumb Code     0  startup_a2fxxxm3.o(.text)
    ACE_Comp11_Rise_IRQHandler               0x000021ff   Thumb Code     0  startup_a2fxxxm3.o(.text)
    ACE_Comp1_Fall_IRQHandler                0x000021ff   Thumb Code     0  startup_a2fxxxm3.o(.text)
    ACE_Comp1_Rise_IRQHandler                0x000021ff   Thumb Code     0  startup_a2fxxxm3.o(.text)
    ACE_Comp2_Fall_IRQHandler                0x000021ff   Thumb Code     0  startup_a2fxxxm3.o(.text)
    ACE_Comp2_Rise_IRQHandler                0x000021ff   Thumb Code     0  startup_a2fxxxm3.o(.text)
    ACE_Comp3_Fall_IRQHandler                0x000021ff   Thumb Code     0  startup_a2fxxxm3.o(.text)
    ACE_Comp3_Rise_IRQHandler                0x000021ff   Thumb Code     0  startup_a2fxxxm3.o(.text)
    ACE_Comp4_Fall_IRQHandler                0x000021ff   Thumb Code     0  startup_a2fxxxm3.o(.text)
    ACE_Comp4_Rise_IRQHandler                0x000021ff   Thumb Code     0  startup_a2fxxxm3.o(.text)
    ACE_Comp5_Fall_IRQHandler                0x000021ff   Thumb Code     0  startup_a2fxxxm3.o(.text)
    ACE_Comp5_Rise_IRQHandler                0x000021ff   Thumb Code     0  startup_a2fxxxm3.o(.text)
    ACE_Comp6_Fall_IRQHandler                0x000021ff   Thumb Code     0  startup_a2fxxxm3.o(.text)
    ACE_Comp6_Rise_IRQHandler                0x000021ff   Thumb Code     0  startup_a2fxxxm3.o(.text)
    ACE_Comp7_Fall_IRQHandler                0x000021ff   Thumb Code     0  startup_a2fxxxm3.o(.text)
    ACE_Comp7_Rise_IRQHandler                0x000021ff   Thumb Code     0  startup_a2fxxxm3.o(.text)
    ACE_Comp8_Fall_IRQHandler                0x000021ff   Thumb Code     0  startup_a2fxxxm3.o(.text)
    ACE_Comp8_Rise_IRQHandler                0x000021ff   Thumb Code     0  startup_a2fxxxm3.o(.text)
    ACE_Comp9_Fall_IRQHandler                0x000021ff   Thumb Code     0  startup_a2fxxxm3.o(.text)
    ACE_Comp9_Rise_IRQHandler                0x000021ff   Thumb Code     0  startup_a2fxxxm3.o(.text)
    ACE_PC0_Flag0_IRQHandler                 0x000021ff   Thumb Code     0  startup_a2fxxxm3.o(.text)
    ACE_PC0_Flag1_IRQHandler                 0x000021ff   Thumb Code     0  startup_a2fxxxm3.o(.text)
    ACE_PC0_Flag2_IRQHandler                 0x000021ff   Thumb Code     0  startup_a2fxxxm3.o(.text)
    ACE_PC0_Flag3_IRQHandler                 0x000021ff   Thumb Code     0  startup_a2fxxxm3.o(.text)
    ACE_PC1_Flag0_IRQHandler                 0x000021ff   Thumb Code     0  startup_a2fxxxm3.o(.text)
    ACE_PC1_Flag1_IRQHandler                 0x000021ff   Thumb Code     0  startup_a2fxxxm3.o(.text)
    ACE_PC1_Flag2_IRQHandler                 0x000021ff   Thumb Code     0  startup_a2fxxxm3.o(.text)
    ACE_PC1_Flag3_IRQHandler                 0x000021ff   Thumb Code     0  startup_a2fxxxm3.o(.text)
    ACE_PC2_Flag0_IRQHandler                 0x000021ff   Thumb Code     0  startup_a2fxxxm3.o(.text)
    ACE_PC2_Flag1_IRQHandler                 0x000021ff   Thumb Code     0  startup_a2fxxxm3.o(.text)
    ACE_PC2_Flag2_IRQHandler                 0x000021ff   Thumb Code     0  startup_a2fxxxm3.o(.text)
    ACE_PC2_Flag3_IRQHandler                 0x000021ff   Thumb Code     0  startup_a2fxxxm3.o(.text)
    BrownOut_1_5V_IRQHandler                 0x000021ff   Thumb Code     0  startup_a2fxxxm3.o(.text)
    BrownOut_3_3V_IRQHandler                 0x000021ff   Thumb Code     0  startup_a2fxxxm3.o(.text)
    CommError_IRQHandler                     0x000021ff   Thumb Code     0  startup_a2fxxxm3.o(.text)
    DMA_IRQHandler                           0x000021ff   Thumb Code     0  startup_a2fxxxm3.o(.text)
    ENVM0_IRQHandler                         0x000021ff   Thumb Code     0  startup_a2fxxxm3.o(.text)
    ENVM1_IRQHandler                         0x000021ff   Thumb Code     0  startup_a2fxxxm3.o(.text)
    EthernetMAC_IRQHandler                   0x000021ff   Thumb Code     0  startup_a2fxxxm3.o(.text)
    Fabric_IRQHandler                        0x000021ff   Thumb Code     0  startup_a2fxxxm3.o(.text)
    GPIO0_IRQHandler                         0x000021ff   Thumb Code     0  startup_a2fxxxm3.o(.text)
    GPIO10_IRQHandler                        0x000021ff   Thumb Code     0  startup_a2fxxxm3.o(.text)
    GPIO11_IRQHandler                        0x000021ff   Thumb Code     0  startup_a2fxxxm3.o(.text)
    GPIO12_IRQHandler                        0x000021ff   Thumb Code     0  startup_a2fxxxm3.o(.text)
    GPIO13_IRQHandler                        0x000021ff   Thumb Code     0  startup_a2fxxxm3.o(.text)
    GPIO14_IRQHandler                        0x000021ff   Thumb Code     0  startup_a2fxxxm3.o(.text)
    GPIO15_IRQHandler                        0x000021ff   Thumb Code     0  startup_a2fxxxm3.o(.text)
    GPIO16_IRQHandler                        0x000021ff   Thumb Code     0  startup_a2fxxxm3.o(.text)
    GPIO17_IRQHandler                        0x000021ff   Thumb Code     0  startup_a2fxxxm3.o(.text)
    GPIO18_IRQHandler                        0x000021ff   Thumb Code     0  startup_a2fxxxm3.o(.text)
    GPIO19_IRQHandler                        0x000021ff   Thumb Code     0  startup_a2fxxxm3.o(.text)
    GPIO1_IRQHandler                         0x000021ff   Thumb Code     0  startup_a2fxxxm3.o(.text)
    GPIO20_IRQHandler                        0x000021ff   Thumb Code     0  startup_a2fxxxm3.o(.text)
    GPIO21_IRQHandler                        0x000021ff   Thumb Code     0  startup_a2fxxxm3.o(.text)
    GPIO22_IRQHandler                        0x000021ff   Thumb Code     0  startup_a2fxxxm3.o(.text)
    GPIO23_IRQHandler                        0x000021ff   Thumb Code     0  startup_a2fxxxm3.o(.text)
    GPIO24_IRQHandler                        0x000021ff   Thumb Code     0  startup_a2fxxxm3.o(.text)
    GPIO25_IRQHandler                        0x000021ff   Thumb Code     0  startup_a2fxxxm3.o(.text)
    GPIO26_IRQHandler                        0x000021ff   Thumb Code     0  startup_a2fxxxm3.o(.text)
    GPIO27_IRQHandler                        0x000021ff   Thumb Code     0  startup_a2fxxxm3.o(.text)
    GPIO28_IRQHandler                        0x000021ff   Thumb Code     0  startup_a2fxxxm3.o(.text)
    GPIO29_IRQHandler                        0x000021ff   Thumb Code     0  startup_a2fxxxm3.o(.text)
    GPIO2_IRQHandler                         0x000021ff   Thumb Code     0  startup_a2fxxxm3.o(.text)
    GPIO30_IRQHandler                        0x000021ff   Thumb Code     0  startup_a2fxxxm3.o(.text)
    GPIO31_IRQHandler                        0x000021ff   Thumb Code     0  startup_a2fxxxm3.o(.text)
    GPIO3_IRQHandler                         0x000021ff   Thumb Code     0  startup_a2fxxxm3.o(.text)
    GPIO4_IRQHandler                         0x000021ff   Thumb Code     0  startup_a2fxxxm3.o(.text)
    GPIO5_IRQHandler                         0x000021ff   Thumb Code     0  startup_a2fxxxm3.o(.text)
    GPIO6_IRQHandler                         0x000021ff   Thumb Code     0  startup_a2fxxxm3.o(.text)
    GPIO7_IRQHandler                         0x000021ff   Thumb Code     0  startup_a2fxxxm3.o(.text)
    GPIO8_IRQHandler                         0x000021ff   Thumb Code     0  startup_a2fxxxm3.o(.text)
    GPIO9_IRQHandler                         0x000021ff   Thumb Code     0  startup_a2fxxxm3.o(.text)
    I2C0_IRQHandler                          0x000021ff   Thumb Code     0  startup_a2fxxxm3.o(.text)
    I2C0_SMBAlert_IRQHandler                 0x000021ff   Thumb Code     0  startup_a2fxxxm3.o(.text)
    I2C0_SMBus_IRQHandler                    0x000021ff   Thumb Code     0  startup_a2fxxxm3.o(.text)
    I2C1_IRQHandler                          0x000021ff   Thumb Code     0  startup_a2fxxxm3.o(.text)
    I2C1_SMBAlert_IRQHandler                 0x000021ff   Thumb Code     0  startup_a2fxxxm3.o(.text)
    I2C1_SMBus_IRQHandler                    0x000021ff   Thumb Code     0  startup_a2fxxxm3.o(.text)
    IAP_IRQHandler                           0x000021ff   Thumb Code     0  startup_a2fxxxm3.o(.text)
    PLL_LockLost_IRQHandler                  0x000021ff   Thumb Code     0  startup_a2fxxxm3.o(.text)
    PLL_Lock_IRQHandler                      0x000021ff   Thumb Code     0  startup_a2fxxxm3.o(.text)
    RTCIF_Pub_IRQHandler                     0x000021ff   Thumb Code     0  startup_a2fxxxm3.o(.text)
    RTC_Match_IRQHandler                     0x000021ff   Thumb Code     0  startup_a2fxxxm3.o(.text)
    SPI0_IRQHandler                          0x000021ff   Thumb Code     0  startup_a2fxxxm3.o(.text)
    SPI1_IRQHandler                          0x000021ff   Thumb Code     0  startup_a2fxxxm3.o(.text)
    Timer1_IRQHandler                        0x000021ff   Thumb Code     0  startup_a2fxxxm3.o(.text)
    Timer2_IRQHandler                        0x000021ff   Thumb Code     0  startup_a2fxxxm3.o(.text)
    WdogWakeup_IRQHandler                    0x000021ff   Thumb Code     0  startup_a2fxxxm3.o(.text)
    __scatterload                            0x00002209   Thumb Code    28  init.o(.text)
    __scatterload_rt2                        0x00002209   Thumb Code     0  init.o(.text)
    __0snprintf$1                            0x0000222d   Thumb Code    36  printf1.o(i.__0snprintf$1)
    __1snprintf$1                            0x0000222d   Thumb Code     0  printf1.o(i.__0snprintf$1)
    __2snprintf                              0x0000222d   Thumb Code     0  printf1.o(i.__0snprintf$1)
    __scatterload_copy                       0x00002255   Thumb Code    14  handlers.o(i.__scatterload_copy)
    __scatterload_null                       0x00002263   Thumb Code     2  handlers.o(i.__scatterload_null)
    __scatterload_zeroinit                   0x00002265   Thumb Code    14  handlers.o(i.__scatterload_zeroinit)
    comp_id_2_scb_lut                        0x00002594   Data          10  mss_ace.o(.constdata)
    g_ace_current_resistors                  0x00002670   Data           8  ace_config.o(.constdata)
    g_ace_external_varef_used                0x00002678   Data           2  ace_config.o(.constdata)
    g_ace_channel_0_name                     0x0000267a   Data          12  ace_config.o(.constdata)
    g_channel_0_flags_lut                    0x00002686   Data           8  ace_config.o(.constdata)
    g_ace_ppe_flag_0_name                    0x0000268e   Data          22  ace_config.o(.constdata)
    g_ace_ppe_flag_1_name                    0x000026a4   Data          22  ace_config.o(.constdata)
    g_ace_ppe_flag_2_name                    0x000026ba   Data          22  ace_config.o(.constdata)
    g_ace_ppe_flag_3_name                    0x000026d0   Data          22  ace_config.o(.constdata)
    g_ace_ppe_transforms_desc_table          0x000026e6   Data           8  ace_config.o(.constdata)
    g_ace_sse_proc_0_name                    0x000026ee   Data          10  ace_config.o(.constdata)
    g_ace_sse_proc_0_sequence                0x000026f8   Data          12  ace_config.o(.constdata)
    g_ace_sse_proc_1_name                    0x00002704   Data          10  ace_config.o(.constdata)
    g_ace_sse_proc_1_sequence                0x0000270e   Data           6  ace_config.o(.constdata)
    Region$$Table$$Base                      0x00002714   Number         0  anon$$obj.o(Region$$Table)
    Region$$Table$$Limit                     0x00002734   Number         0  anon$$obj.o(Region$$Table)
    SystemFrequency                          0x2000000c   Data           4  system_a2fxxxm3.o(.data)
    SystemCoreClock                          0x20000010   Data           4  system_a2fxxxm3.o(.data)
    g_FrequencyPCLK0                         0x20000014   Data           4  system_a2fxxxm3.o(.data)
    g_FrequencyPCLK1                         0x20000018   Data           4  system_a2fxxxm3.o(.data)
    g_FrequencyACE                           0x2000001c   Data           4  system_a2fxxxm3.o(.data)
    g_FrequencyFPGA                          0x20000020   Data           4  system_a2fxxxm3.o(.data)
    g_ace_adc_config                         0x20000024   Data           8  ace_config.o(.data)
    g_ace_channel_desc_table                 0x2000002c   Data          16  ace_config.o(.data)
    g_ppe_flags_desc_table                   0x2000003c   Data          64  ace_config.o(.data)
    g_sse_sequences_desc_table               0x2000007c   Data          40  ace_config.o(.data)
    g_mss_uart0                              0x200003d0   Data          40  mss_uart.o(.bss)
    g_mss_uart1                              0x200003f8   Data          40  mss_uart.o(.bss)
    __initial_sp                             0x20001420   Data           0  startup_a2fxxxm3.o(STACK)



==============================================================================

Memory Map of the image

  Image Entry point : 0x00000299

  Load Region LR_ROM1 (Base: 0x00000000, Size: 0x000027d8, Max: 0x01000000, ABSOLUTE)

    Execution Region ER_ROM1 (Base: 0x00000000, Size: 0x00002734, Max: 0x01000000, ABSOLUTE)

    Base Addr    Size         Type   Attr      Idx    E Section Name        Object

    0x00000000   0x00000298   Data   RO          553    RESET               Voltage_Monitor_MSS_MSS_CM3_0_hw_platform.lib(startup_a2fxxxm3.o)
    0x00000298   0x00000000   Code   RO          258  * .ARM.Collect$$$$00000000  mc_w.l(entry.o)
    0x00000298   0x00000004   Code   RO          528    .ARM.Collect$$$$00000001  mc_w.l(entry2.o)
    0x0000029c   0x00000004   Code   RO          531    .ARM.Collect$$$$00000004  mc_w.l(entry5.o)
    0x000002a0   0x00000008   Code   RO          532    .ARM.Collect$$$$00000007  mc_w.l(entry7.o)
    0x000002a8   0x00000004   Code   RO          529    .ARM.Collect$$$$00002712  mc_w.l(entry2.o)
    0x000002ac   0x000001b8   Code   RO            1    .text               main.o
    0x00000464   0x00000564   Code   RO           52    .text               Voltage_Monitor_MSS_MSS_CM3_0_hw_platform.lib(ace_convert.o)
    0x000009c8   0x00000930   Code   RO           98    .text               Voltage_Monitor_MSS_MSS_CM3_0_hw_platform.lib(ace_flags.o)
    0x000012f8   0x0000059c   Code   RO          122    .text               Voltage_Monitor_MSS_MSS_CM3_0_hw_platform.lib(mss_ace.o)
    0x00001894   0x0000019c   Code   RO          144    .text               Voltage_Monitor_MSS_MSS_CM3_0_hw_platform.lib(mss_gpio.o)
    0x00001a30   0x00000614   Code   RO          175    .text               Voltage_Monitor_MSS_MSS_CM3_0_hw_platform.lib(mss_uart.o)
    0x00002044   0x00000130   Code   RO          207    .text               Voltage_Monitor_MSS_MSS_CM3_0_hw_platform.lib(system_a2fxxxm3.o)
    0x00002174   0x00000024   Code   RO          261    .text               mc_w.l(memcpya.o)
    0x00002198   0x0000001e   Code   RO          263    .text               mc_w.l(strncmp.o)
    0x000021b6   0x0000002c   Code   RO          536    .text               mc_w.l(uidiv.o)
    0x000021e2   0x00000002   PAD
    0x000021e4   0x00000024   Code   RO          554    .text               Voltage_Monitor_MSS_MSS_CM3_0_hw_platform.lib(startup_a2fxxxm3.o)
    0x00002208   0x00000024   Code   RO          559    .text               mc_w.l(init.o)
    0x0000222c   0x00000028   Code   RO          313    i.__0snprintf$1     mc_w.l(printf1.o)
    0x00002254   0x0000000e   Code   RO          573    i.__scatterload_copy  mc_w.l(handlers.o)
    0x00002262   0x00000002   Code   RO          574    i.__scatterload_null  mc_w.l(handlers.o)
    0x00002264   0x0000000e   Code   RO          575    i.__scatterload_zeroinit  mc_w.l(handlers.o)
    0x00002272   0x00000002   PAD
    0x00002274   0x00000150   Code   RO          319    i._printf_core      mc_w.l(printf1.o)
    0x000023c4   0x00000016   Code   RO          320    i._snputc           mc_w.l(printf1.o)
    0x000023da   0x000000cc   Data   RO           54    .constdata          Voltage_Monitor_MSS_MSS_CM3_0_hw_platform.lib(ace_convert.o)
    0x000024a6   0x00000002   PAD
    0x000024a8   0x000000b0   Data   RO          100    .constdata          Voltage_Monitor_MSS_MSS_CM3_0_hw_platform.lib(ace_flags.o)
    0x00002558   0x00000046   Data   RO          123    .constdata          Voltage_Monitor_MSS_MSS_CM3_0_hw_platform.lib(mss_ace.o)
    0x0000259e   0x00000002   PAD
    0x000025a0   0x000000c0   Data   RO          145    .constdata          Voltage_Monitor_MSS_MSS_CM3_0_hw_platform.lib(mss_gpio.o)
    0x00002660   0x00000010   Data   RO          208    .constdata          Voltage_Monitor_MSS_MSS_CM3_0_hw_platform.lib(system_a2fxxxm3.o)
    0x00002670   0x000000a4   Data   RO          236    .constdata          Voltage_Monitor_MSS_MSS_CM3_0_hw_platform.lib(ace_config.o)
    0x00002714   0x00000020   Data   RO          571    Region$$Table       anon$$obj.o


    Execution Region RW_IRAM1 (Base: 0x20000000, Size: 0x00001420, Max: 0x00010000, ABSOLUTE)

    Base Addr    Size         Type   Attr      Idx    E Section Name        Object

    0x20000000   0x00000001   Data   RW           55    .data               Voltage_Monitor_MSS_MSS_CM3_0_hw_platform.lib(ace_convert.o)
    0x20000001   0x00000003   PAD
    0x20000004   0x00000008   Data   RW          101    .data               Voltage_Monitor_MSS_MSS_CM3_0_hw_platform.lib(ace_flags.o)
    0x2000000c   0x00000018   Data   RW          209    .data               Voltage_Monitor_MSS_MSS_CM3_0_hw_platform.lib(system_a2fxxxm3.o)
    0x20000024   0x00000080   Data   RW          237    .data               Voltage_Monitor_MSS_MSS_CM3_0_hw_platform.lib(ace_config.o)
    0x200000a4   0x0000000a   Zero   RW           53    .bss                Voltage_Monitor_MSS_MSS_CM3_0_hw_platform.lib(ace_convert.o)
    0x200000ae   0x00000002   PAD
    0x200000b0   0x00000320   Zero   RW           99    .bss                Voltage_Monitor_MSS_MSS_CM3_0_hw_platform.lib(ace_flags.o)
    0x200003d0   0x00000050   Zero   RW          176    .bss                Voltage_Monitor_MSS_MSS_CM3_0_hw_platform.lib(mss_uart.o)
    0x20000420   0x00001000   Zero   RW          551    STACK               Voltage_Monitor_MSS_MSS_CM3_0_hw_platform.lib(startup_a2fxxxm3.o)


==============================================================================

Image component sizes


      Code (inc. data)   RO Data    RW Data    ZI Data      Debug   Object Name

       440        108          0          0          0       8487   main.o

    ----------------------------------------------------------------------
       440        108         32          0          0       8487   Object Totals
         0          0         32          0          0          0   (incl. Generated)
         0          0          0          0          0          0   (incl. Padding)

    ----------------------------------------------------------------------

      Code (inc. data)   RO Data    RW Data    ZI Data      Debug   Library Member Name

         0          0        164        128          0       9523   ace_config.o
      1380         68        204          1         10      37092   ace_convert.o
      2352         86        176          8        800      33745   ace_flags.o
      1436         98         70          0          0       9775   mss_ace.o
       412         32        192          0          0      42264   mss_gpio.o
      1556         48          0          0         80      47893   mss_uart.o
        36          8        664          0       4096        816   startup_a2fxxxm3.o
       304         72         16         24          0       3070   system_a2fxxxm3.o
         0          0          0          0          0          0   entry.o
         8          4          0          0          0          0   entry2.o
         4          0          0          0          0          0   entry5.o
         8          4          0          0          0          0   entry7.o
        30          0          0          0          0          0   handlers.o
        36          8          0          0          0         68   init.o
        36          0          0          0          0         68   memcpya.o
       398          8          0          0          0        248   printf1.o
        30          0          0          0          0         80   strncmp.o
        44          0          0          0          0         80   uidiv.o

    ----------------------------------------------------------------------
      8074        436       1490        164       4988     184722   Library Totals
         4          0          4          3          2          0   (incl. Padding)

    ----------------------------------------------------------------------

      Code (inc. data)   RO Data    RW Data    ZI Data      Debug   Library Name

      7476        412       1486        161       4986     184178   Voltage_Monitor_MSS_MSS_CM3_0_hw_platform.lib
       594         24          0          0          0        544   mc_w.l

    ----------------------------------------------------------------------
      8074        436       1490        164       4988     184722   Library Totals

    ----------------------------------------------------------------------

==============================================================================


      Code (inc. data)   RO Data    RW Data    ZI Data      Debug   

      8514        544       1522        164       4988     192377   Grand Totals
      8514        544       1522        164       4988     192377   ELF Image Totals
      8514        544       1522        164          0          0   ROM Totals

==============================================================================

    Total RO  Size (Code + RO Data)                10036 (   9.80kB)
    Total RW  Size (RW Data + ZI Data)              5152 (   5.03kB)
    Total ROM Size (Code + RO Data + RW Data)      10200 (   9.96kB)

==============================================================================

